:1000000005280000000000000629831285018316E0
:10001000003085008312860183160330860000308D
:10002000A8000A30A70064008316503081008312B4
:100030000301AA008120F6302006031D1A280301BF
:100040002106031D1A2818089000190891001A307B
:10005000A30090308B00A308031D2B2800308B00D9
:100060008E20F5302006031D1A2803012106031DEA
:100070001A2818089200190893001A30A30090302B
:100080008B00A308031D412800308B008E20973081
:10009000200603194F28F3302006031D1A280301F8
:1000A0002106031D1A2818089400190895001A3013
:1000B000A30090308B00A308031D5B2800308B0049
:1000C0008E2096302006031D1A2803012106031DE9
:1000D0001A2818089600190897001208F039003AF3
:1000E000031D1A2813080339A600A60D3030260771
:1000F000840016088000840A1708800030088600F3
:100100001A28061C812886208E20080003108618D5
:1001100003149B0D9A0D990D980D08001A30A40038
:10012000A001A1011B089F001A089E0019089D004C
:1001300018089C009F0D9E0D9D0D9C0D031CA92869
:100140002408B220A0062408CE20A106A40B9A28D9
:1001500008000330AE20A40B9A280800A500A50BC8
:10016000AF28080082070000C634E334A9343D34C8
:100170007B34F73480346E34DD34D534C434E73422
:10018000A1342D345B34B7340034003401340234EC
:1001900004340834103420344034803482070000A2
:1001A000C034C034C034C034803400344034C0342F
:1001B00080344034C034C034C034C034803400345F
:1001C00040348034003400340034003400340034CF
:1001D000003400343008FB203108FB203208FB20BB
:1001E0003308FB203408FB203508FB203608FB20B1
:1001F0003708FB200800AB002A08031DFC282B0849
:10020000A9001030AA00A0308B000800AC00030E3B
:10021000AD008B1C0F298620A3038B100900061943
:100220001B290310A90D031C1829861506151C2966
:10023000861106151C290611AA0B20298B122029CC
:10024000280881000B1109002D0E8300AD0E2D0E24
:1002500009002A29380881000B110900000000005C
:10026000000000000000000000000000000000008E
:10027000000000000000000000000000000000007E
:10028000000000000000000000000000000000006E
:10029000000000000000000000000000000000005E
:02400E00F13F80
:1042000000000000000000000000000000000000AE
:10421000000000000000000000000000000000009E
:10422000000000000000000000000000000000008E
:10423000000000000000000000000000000000007E
:10424000000000000000000000000000000000006E
:10425000000000000000000000000000000000005E
:10426000000000000000000000000000000000004E
:10427000000000000000000000000000000000003E
:00000001FF
